:100000007FC0000099C0000097C0000095C00000AC
:1000100093C0000091C000008FC000008DC00000A0
:100020008BC0000089C0000087C00000D3C400005E
:1000300073C5000081C000007FC000007DC00000CB
:100040007BC0000079C0000077C0000075C00000D0
:1000500073C0000071C000006FC000006DC00000E0
:100060006BC0000069C0000067C0000065C00000F0
:1000700063C000001C034C005500460041002000F6
:100080004300440043002000440065006D006F0001
:10009000000018034400650061006E00200043006A
:1000A00061006D0065007200610000000403090436
:1000B00009023E00020100C03209040000010202F0
:1000C0000100052400100104240206052406000195
:1000D000070582030800FF09040100020A0000006E
:1000E0000705040210000507058302100005120130
:1000F000100102000008EB03442001000102DC01B2
:1001000011241FBECFEFD2E0DEBFCDBF11E0A0E0D3
:10011000B1E0E0E8F1E102C005900D92AC31B10729
:10012000D9F721E0ACE1B1E001C01D92A034B207E3
:10013000E1F7C0D70C94BE0863CF292F33272230B4
:10014000310559F02330310569F02130310521F5B1
:1001500082E190E02EEE30E028C08EE390E020EBCC
:1001600030E023C099278130910551F018F00297B3
:1001700069F017C0ECEAF0E0849190E09F0115C0AF
:10018000E2E9F0E0849190E09F010FC0E4E7F0E045
:10019000849190E09F0109C080E090E020E030E091
:1001A00004C080E090E020E030E0FA013183208359
:1001B0000895CF93DF93EC01FC0170968BE0DF0193
:1001C0001D928A95E9F782E08C83898783E08E8788
:1001D00061E0CE01019608D3882351F061E0CE01A1
:1001E000069602D3882321F061E0CE010B96FCD263
:1001F000DF91CF910895CF93FC0190912E0194301F
:10020000E9F484899589A689B789892B8A2B8B2B58
:10021000B9F0C62F81818F708093E9008091E8004A
:1002200085FD08C0E8EEF0E080818E7780834FD3B3
:10023000811107C0C093F10080E003C082E001C0DB
:1002400082E0CF910895FB01682F84859585D3DFE7
:1002500021E030E0811102C020E030E088279927BA
:10026000821B930B0895FC0190912E01943009F5A7
:1002700084899589A689B789892B8A2B8B2BD9F0FC
:1002800081818F708093E9008091F2008823B1F022
:10029000E8EEF0E0908180818E77808395FD0DC03F
:1002A00016D381110BC0E8EEF0E090819E77908329
:1002B000089582E0089582E0089580E00895FC01A9
:1002C00090912E01943091F484899589A689B789FB
:1002D000892B8A2B8B2B51F081818F708093E900C1
:1002E0008091E80080FF02C0CF01BDCF0895FC01DE
:1002F00090912E01943001F584899589A689B7895A
:10030000892B8A2B8B2BD9F086818F708093E90003
:100310008091E80082FF16C08091F200811108C030
:10032000E8EEF0E080818B77808380E090E00895B4
:100330008091F20090E0089580E090E0089580E0E0
:1003400090E0089580E090E0089520912E012430FF
:1003500039F5FC014489558966897789452B462BF7
:10036000472B09F186818F708093E9008091E80026
:1003700082FF1CC08091F200882321F02091F100BF
:1003800030E002C02FEF3FEF8091F200811111C0E9
:10039000E8EEF0E080818B778083822F932F0895A1
:1003A0008FEF9FEF08958FEF9FEF08958FEF9FEFEF
:1003B0000895822F932F0895FC0184859585C5DFCC
:1003C000992314F48EEF9FEF0895FB012EE0DB01DB
:1003D0001D922A95E9F723E0238323E231E0318758
:1003E00020872CED31E03387228795878487089515
:1003F0000895CF93DF93FC019091E80093FF96C09E
:10040000208130E08091330190913401821793076D
:1004100009F08CC0EF0180913001813259F018F45D
:100420008032B9F183C0823209F45FC0833209F4AB
:100430006FC07CC080912F01813A09F077C0E8EE4F
:10044000F0E08081877F8083808180FFFDCF8C8971
:100450009D89AE89BF89E1EFF0E08083492F5A2F53
:100460006B2F77274083AD016627772740838B2F3B
:100470009927AA27BB278083888D8083898D8083D5
:100480008A8D8083E8EEF0E080818E778083FBD1D7
:100490004DC080912F01813209F048C0E8EEF0E0B4
:1004A0008081877F808305C080912E01882309F495
:1004B0003DC0808182FFF8CFE1EFF0E03081208104
:1004C000908180813C8B2D8B9E8B8F8B8081888F40
:1004D0008081898F80818A8FE8EEF0E080818B7740
:1004E0008083D1D1CE0184DF21C080912F01813260
:1004F000E9F4E8EEF0E08081877F8083C4D18091C9
:10050000310190913201998B888BCE0136D60EC085
:1005100080912F01813251F4E8EEF0E08081877FF5
:100520008083B1D160913101CE0162DFDF91CF9143
:100530000895EF92FF921F93CF93DF93209135019F
:10054000309136012617370758F06115710539F4D7
:10055000E8EEF0E020812E7720839B0101C09B0113
:10056000A82FB92F40E0E8EEF0E062EF70E00F2E28
:10057000F1EFEF2EF12CF02D51E010E02BC0809127
:100580002E018823F1F18530F1F1808183FD3DC09A
:10059000808182FD2FC0808180FF1CC0EB0188819B
:1005A00090E02115310579F08830910560F44D9186
:1005B000E70148832150310901962115310519F0D1
:1005C00088309105A1F7452F089709F0412F8081C8
:1005D0008E7780832115310591F64111D0CF0AC065
:1005E00080912E01882399F0853099F0808183FFD6
:1005F00003C011C0E8EEF0E0808182FFF1CF80E01F
:100600000BC082E009C083E007C081E005C082E042
:1006100003C083E001C081E0DF91CF911F91FF9083
:10062000EF900895EF92FF921F93CF93DF93209165
:100630003501309136012617370758F061157105DD
:1006400039F4E8EEF0E020812E7720839B0101C091
:100650009B01E82FF92F60E0A8EEB0E042EF50E0F8
:100660000F2EF1EFEF2EF12CF02D71E010E02EC0E7
:1006700080912E01882309F440C0853009F43FC0E1
:100680008C9183FD3EC08C9182FD30C08C9180FFA7
:100690001DC0EA01888190E02115310581F0883084
:1006A000910568F46491E70168833196215031091E
:1006B00001962115310519F08830910599F7672FBA
:1006C000089709F0612F8C918E778C932115310555
:1006D00079F66111CDCF0AC080912E01882399F05F
:1006E000853099F0808183FF03C011C0E8EEF0E00F
:1006F000808182FFF1CF80E00BC082E009C083E0FF
:1007000007C081E005C082E003C083E001C081E052
:10071000DF91CF911F91FF90EF9008958F929F925C
:10072000BF92CF92DF92EF92FF920F931F93CF93DE
:10073000DF93853070F126C0292F2F70E7012883C1
:10074000891731F0E80178812081E401588103C0E4
:10075000242F762F5B2D21FF12C03C913E7F3C93CE
:1007600030813D7F30833C9131603C93E801788358
:100770002083E4015883E6012881222344F49F5F0B
:100780009530D1F68F708093E90081E021C080E040
:100790001FC0982F9F709093E900982F242F762FD9
:1007A00050E0ABEEB0E0EDEEF0E00CEE10E00F2E1E
:1007B000F0EF8F2E912CF02D0F2EFEEECF2ED12CA0
:1007C000F02D0F2EF9EEEF2EF12CF02DB12CC3CF22
:1007D000DF91CF911F910F91FF90EF90DF90CF901D
:1007E000BF909F908F900895EF92FF920F931F9369
:1007F000CF93DF936623E9F1062FC82FD92F10E09E
:100800000F2EF6E0FF2EF02D6894EE24E1F85881CB
:10081000552349F19C81E981FA816B81852F8F7085
:10082000853048F5923010F44E2D01C04F2DE9303F
:10083000F10550F028E030E090E09F5F220F331F79
:100840002E173F07D0F301C090E09295907F492B7F
:100850006295660F660F607C551F5527551F652BE7
:100860005DDF882349F01F5F25960113D0CF81E01B
:1008700003C081E001C080E0DF91CF911F910F9113
:10088000FF90EF90089580912F01882344F0E8EEC7
:10089000F0E014C080912E01811103C00895E8EEAC
:1008A000F0E0808182FFF6CFE8EEF0E080818B7788
:1008B0008083089580912E01882341F0808180FFFC
:1008C000F9CFE8EEF0E080818E77808308950F9372
:1008D0001F93CF93DF932091E4003091E50065E60C
:1008E000ACEEB0E0E8EEF0E00BEE10E044EE50E0ED
:1008F00001C09C019C91892F817090FD1DC020C07A
:1009000080912E01882381F0853081F0E801888173
:1009100085FD0EC0EA01888199812817390751F3B6
:10092000615039F784E00FC082E00DC083E00BC056
:1009300081E009C080E007C0808180FFE1CFFACF6D
:10094000908192FFDDCFDF91CF911F910F9108959C
:100950003BD03DD0E8EDF0E080818F7780838081CF
:100960008068808380818F7D808319BC82E089BD0F
:1009700009B400FEFDCF10922E0110922A011092B0
:100980002C0110922B0142E060E080E0C7DEE1EE36
:10099000F0E080818E7F8083E2EEF0E080818160F4
:1009A0008083808188608083E0EEF0E080818E7FAC
:1009B00080830895E3E6F0E080818E7F808381E08C
:1009C00080932D01C5CF08951092E20008951092F2
:1009D000E10008951F920F920FB60F9211242F93EA
:1009E0003F934F935F936F937F938F939F93AF93B7
:1009F000BF93EF93FF938091E10082FF0AC0809143
:100A0000E20082FF06C0E1EEF0E080818B7F808310
:100A10004BD28091E10080FF15C08091E20080FF01
:100A200011C0E2EEF0E080818E7F80838081806162
:100A30008083E8EDF0E080818062808319BC1092B1
:100A40002E0192D38091E10084FF2EC08091E200BC
:100A500084FF2AC019BC82E089BD09B400FEFDCF25
:100A6000E8EDF0E080818F7D8083E1EEF0E0808131
:100A70008F7E8083E2EEF0E080818F7E80838081B4
:100A80008160808380912A01882321F084E0809313
:100A90002E0109C08091E300882314F081E001C099
:100AA00083E080932E015FD38091E10083FF23C018
:100AB0008091E20083FF1FC0E1EEF0E08081877F3C
:100AC000808382E080932E0110922A0180818E7FA4
:100AD0008083E2EEF0E080818E7F80838081806180
:100AE000808342E060E080E019DEE0EFF0E08081AA
:100AF00088608083D9D1FF91EF91BF91AF919F9191
:100B00008F917F916F915F914F913F912F910F90B6
:100B10000FBE0F901F9018951F920F920FB60F9255
:100B20001124EF92FF920F931F932F933F934F93B4
:100B30005F936F937F938F939F93AF93BF93CF9365
:100B4000DF93EF93FF93C091E900CF708091EC00A9
:100B5000D82FD17080FDD0E80F2EF9EEEF2EF12CBA
:100B6000F02DF701108200EF10E0F8018081877FFF
:100B70008083789421D0F7011082F8018081886009
:100B80008083CD2BCF70F701C083FF91EF91DF9170
:100B9000CF91BF91AF919F918F917F916F915F9115
:100BA0004F913F912F911F910F91FF90EF900F90D8
:100BB0000FBE0F901F9018950F931F93CF93DF9345
:100BC000CDB7DEB7AA970FB6F894DEBF0FBECDBF84
:100BD000EFE2F1E027E331E0A1EFB0E08C91819307
:100BE0002E173F07D9F7C5D28091E80083FF37C1A0
:100BF000EFE2F1E090818181853009F47FC030F42B
:100C00008130C9F168F08330B1F129C1883009F42D
:100C1000F1C0893009F4FEC0863009F020C191C0CE
:100C2000903821F0923809F01AC108C080912B0148
:100C300090912C01992389F082600FC0809133013B
:100C40008F70853008F00BC1E9EEF0E08083809171
:100C5000EB0085FB882780F91082E8EEF0E09081B8
:100C6000977F9083A1EFB0E08C931C9280818E7768
:100C7000808309DEF4C0992309F400C1923009F0A1
:100C8000EEC001C191E0833009F090E090932C0117
:100C90002CC0809133018F709FEF980F943008F033
:100CA000DEC08093E9009091EB0090FF1EC0909110
:100CB0003001933031F4EBEEF0E08081806280838C
:100CC00014C0EBEEF0E090819061908321E030E081
:100CD000A90102C0440F551F8A95E2F7AAEEB0E0C1
:100CE0004C931C928081886080831092E900E8EE2A
:100CF000F0E08081877F8083C6DDB1C09111AFC0F5
:100D0000109131011F77E3EEF0E080818078812B34
:100D10008083E8EEF0E08081877F8083B4DDE8EEB9
:100D2000F0E0808180FFFDCFE3EEF0E0808180681D
:100D30008083111102C082E001C083E080932E0104
:100D40008EC09058923008F08AC080913101909105
:100D500032018C3D53E0950799F583E08A838AE25E
:100D600089835FB7F894DE01139620E03EE041E20C
:100D7000E32FF0E040935700849120FF03C0829559
:100D80008F703F5F8F708A3018F090E0C79602C076
:100D900090E0C0968D939D932F5F243149F75FBFFC
:100DA00008EE10E0F8018081877F80836AE270E0BE
:100DB000CE010196BEDBF80180818B7780834FC026
:100DC0006091330170913401AE014F5F5F4FB5D92F
:100DD000BC01892B09F443C008EE10E0F8019081B2
:100DE000977F908389819A811DDCF80180818B77C0
:100DF000808335C0903899F5E8EEF0E08081877FF8
:100E0000808380912A018093F10080818E77808396
:100E10003ADD25C0911123C08091310190913201BA
:100E200099270297E4F4E8EEF0E08081877F8083E1
:100E30008091310180932A0126DD80912A01882347
:100E400021F084E080932E0109C08091E300882383
:100E500014F081E001C084E080932E0186D180915E
:100E6000E80083FF16C0E8EEF0E08081877F808392
:100E7000EBEEF0E08081806280830BC090913101C5
:100E8000913069F7FFCE80913101882309F401CFB9
:100E90002CCFAA960FB6F894DEBF0FBECDBFDF9160
:100EA000CF911F910F9108950895CF9380912E01B6
:100EB000882399F0C091E900CF708091EC00982FC1
:100EC000917080FD90E8C92B1092E9008091E800B4
:100ED00083FD72DECF70C093E900CF910895FC01CD
:100EE0009081862F809598239083ADECB0E0119788
:100EF000F1F700C0000040FF04C09081962B908362
:100F000003C0908198239083ADECB0E01197F1F786
:100F100000C0000041FF04C09081962B908303C065
:100F2000908198239083ADECB0E01197F1F700C069
:100F3000000042FF04C09081962B908303C09081F3
:100F400098239083ADECB0E01197F1F700C000005A
:100F500043FF04C09081962B908303C09081982317
:100F60009083ADECB0E01197F1F700C0000044FFB2
:100F700004C09081962B908303C090819823908326
:100F8000ADECB0E01197F1F700C0000045FF04C0E0
:100F90009081962B908303C0908198239083ADEC31
:100FA000B0E01197F1F700C0000046FF04C0908147
:100FB000962B908303C0908198239083ADECB0E092
:100FC0001197F1F700C00000442324F48081862BA0
:100FD000808303C09081892380838DEC90E001970A
:100FE000F1F700C000008081682B6083ADECB0E0B9
:100FF0001197F1F700C000008DEC90E00197F1F738
:1010000000C000000895813311F42C9A01C02C987F
:1010100080E090E00895EF92FF920F931F93CF939B
:10102000DF9300D000D000D0CDB7DEB790E8998331
:1010300024EA2A839E838B836C831D828E010F5F3B
:101040001F4F7E0187E0E80EF11CF80141918F01EE
:1010500062E08BE290E043DF0E151F05B1F780E000
:1010600090E026960FB6F894DEBF0FBECDBFDF919D
:10107000CF911F910F91FF90EF90089584B7877FD4
:1010800084BF0FB6F894A895809160008861809322
:101090006000109260000FBE90E080E80FB6F894F8
:1010A00080936100909361000FBE249A83DC599A6B
:1010B000519A0895CF93DF93CDB7DEB72C970FB633
:1010C000F894DEBF0FBECDBFD9DF6CE171E080E0E8
:1010D00091E07BD97894E7E3F1E08FEF848313828A
:1010E0001582818384E68083128210E080E091E0A3
:1010F000FED8892B99F1163009F410E080E091E0D8
:1011000024D9FE013196E10FF11DE10FF11D91830C
:1011100080831F5F89819A8180389105F9F48B81E2
:101120009C81843A9105D1F48B859C85803891050A
:10113000A9F40D811E81C8010197029740F4013086
:10114000110511F48F815FDF6F81802F64DF1A82B8
:1011500019821C821B821C861B8610E080E091E0B5
:10116000AED8A3DEC3CF0895089580E091E021C8F2
:10117000089580E091E03DC908950895F894FFCF67
:10118000008310000001041000000182080000012B
:0C11900000000000000000000000000053
:00000001FF
